:020000040800F2
:10000000001800200508000835050008390500081B
:1000100000000000000000000000000000000000E0
:10002000000000000000000000000000350500088E
:10003000000000000000000035050008350500083C
:1000400035050008350500083505000835050008A8
:100050003505000835050008350500083505000898
:100060003505000835050008350500083505000888
:100070003505000835050008350500083505000878
:100080003505000835050008350500083505000868
:100090003505000835050008350500083505000858
:1000A0003505000835050008350500083505000848
:1000B00035050008350500083505000899010008D8
:1000C000284B10B51A88284B12041B881A43274B5B
:1000D000198849084900885A254908801988023139
:1000E00089B21980198849084900885A214908802D
:1000F0001988023189B21980198849084900885A3B
:100100001D49088019881D48023189B21980198853
:1001100049084900895A1A4A11801A881949023235
:1001200092B21A801C880288944213D902881C88D3
:100130000832121B92B20A80028892B21A801249C7
:10014000124B0A881343124A1A40302353409BB281
:100150000B8010BD0F4804881A889442E6D3082308
:100160000B80ECE70C6000400A6000400460004037
:100170004C6000404E600040506000400260004013
:10018000526000401A600040005C00408080FFFF29
:10019000BF8FFFFF006000409449F8B50B88944C76
:1001A000002B3AD00A88934B9A4234D1002302257F
:1001B000914A924F1380924A1380924A1380924A36
:1001C0001380924A1380924AD08FA843D087D08F51
:1001D000013DA843D0878F481735FB8705808E489F
:1001E000343505808D480835058080258C486D01A3
:1001F000058080258B4805808020FB878A4B000680
:1002000023808A4B18608023D08FDB000343D38781
:10021000874B884A1A8000230B8023881BB2002B4F
:1002200000DBC4E02388844A774F134080221343C5
:10023000238023881B0500D49CE0804D7F232A78EF
:1002400011009943714B1980E9886B4B198000218B
:100250006C4B19803B88FF318B4313433B806023F9
:100260001A4208D08022764B12051B8828009B1862
:100270009847634B188060232A78134052B2002AB3
:100280004DDA002B14D16A78062A0FD16A88110A38
:1002900002291AD003291BD0012920D1694B12262B
:1002A000694A99B21180694A1B0C1380544B1E8015
:1002B0002288674B1343674A1A40C0239B0153406F
:1002C0009BB22380FFF7FCFE47E05E4B1233E6E76C
:1002D000D2B2012A0FD0002A03D0022A15D01E0064
:1002E000E4E7584B584A243399B21180574A1B0C03
:1002F00013800426DAE7534B534A283399B211800E
:10030000524A1B0C1380544ED0E74E4B4E4A7C335E
:1003100099B211804D4A1B0C1380504EC6E7002B3A
:1003200009D16B78052B06D13A886B88D2B21B02B3
:1003300013439BB23B8000212388494A1340494A1A
:1003400013439BB22380484B198023881A43474BA1
:100350001A40474B5A4092B22280284BDB8F5B05F4
:1003600007D580222F4B1A800023244AD3872E4B97
:100370002380F8BD60213B880B40402BEDD13B88AA
:100380001342EAD1264A3B4B2C481B881188802215
:1003900012059B18C9B298472288324B13432D4A45
:1003A0001A40C0239B0153409BB22380D5E7802293
:1003B00023881342D1D023882F490B408021090282
:1003C0000B432380114B1B88934200D17AE7FF2017
:1003D0000D4B19888143C0D01988090A0A43114975
:1003E0000A801A8802401A80B7E7C0460E600040B3
:1003F000005C00403CA5000000600040065C00403E
:100400000260004004600040066000400860004058
:10041000025C0040505C0040186000401C600040DE
:100420001E6000404C5C00402032000000E100E013
:10043000585C00400080FFFF8F0F000054600040B8
:10044000106000407C0400080A6000400C6000401E
:100450008081FFFF8FBFFFFF2A0300001E03000003
:100460008F8EFFFF8080FFFF1A600040BFBFFFFF3D
:1004700030300000126000400F8FFFFF12010002B9
:10048000FF000008C016DC0503020102000109029A
:100490001200010100803209040000000000000089
:1004A000040309042A0349006E00660069006E0017
:1004B0006900740065004E00650073004C0069001F
:1004C0007600650073002E0063006F006D00000071
:1004D000000000000000000000000000000000001C
:1004E000000000000000000000000000000000000C
:1004F00000000000000000001E0349004E004C00F8
:10050000200052006500740072006F002D00500042
:1005100072006F0067000000000000000000000093
:1005200000000000000000000000000000000000CB
:1005300000000000FEE7FFFF004801E02301ADDE00
:10054000FEE7C04602B4714649084900095C49000B
:100550008E4402BC7047C046411D000000616561C9
:1005600062690001130000000536532D4D00060C92
:10057000074D09011901FFFF03B471464908400006
:100580004900095A49008E4403BC7047411D0000D0
:100590000061656162690001130000000536532D9A
:1005A0004D00060C074D09011901FFFF70470A4B6A
:1005B0000A4A10B55A600A4A5A600122DC6814429D
:1005C000FCD11A6101220180D9681142FCD120229C
:1005D000DA6060321A6110BD0020024023016745D5
:1005E000AB89EFCDFF2370B53C4C23804378C588A1
:1005F000102B00D06FE0C37881888078384E0138A6
:100600007269082800D964E0FFF79CFF0563632B3B
:100610003B3149515F008B1E8E227D2B19D8314B07
:100620007360314B73600123F2681A42FCD10223DC
:100630003361802389021B05C9184223716133612C
:10064000C046413BF2681A40FCD12023F36060337E
:1006500033612270254BA2B2240CE8B25A819C81EE
:1006600070BD58001018FFF7A2FF0022F1E78E229C
:10067000012BEED8180480231B05C01840181C4914
:10068000F1E7042363707369A37073691B0AE37055
:1006900073691B0C237173691B0E6371E5E70223F9
:1006A00063701388A37013881B0AE370DDE78E2242
:1006B000012BCED880221B0412059B185918022347
:1006C00063700B88A3700B88EEE70A4B0A4ADA6066
:1006D000CBE78B22BDE780232370BBE7F806002021
:1006E0000020024023016745AB89EFCD0060004048
:1006F000FFFF000000ED00E00400FA05FFFFFFFF30
:10070000FFFFFFFFFFFFFFFFFFFFFFFFFFFFFFFFF9
:10071000FFFFFFFFFFFFFFFFFFFFFFFFFFFFFFFFE9
:10072000FFFFFFFFFFFFFFFFFFFFFFFFFFFFFFFFD9
:10073000FFFFFFFFFFFFFFFFFFFFFFFFFFFFFFFFC9
:10074000FFFFFFFFFFFFFFFFFFFFFFFFFFFFFFFFB9
:10075000FFFFFFFFFFFFFFFFFFFFFFFFFFFFFFFFA9
:10076000FFFFFFFFFFFFFFFFFFFFFFFFFFFFFFFF99
:10077000164B174A9BB21382164B9BB253826846A4
:100780001C300F4A0F4B0430043001681140C91A65
:10079000FAD1094A094B043801681140C91AF2D14B
:1007A0007B460A3303600438013303600CE00A4BD4
:1007B0000A4A1A60FBE7C0460000FFFF000000087D
:1007C000FFFFFF0F0000000100207047E505000853
:1007D00000600040AD05000800300040AAAA0000FB
:1007E000FFFFFFFFFFFFFFFFFFFFFFFFFFFFFFFF19
:1007F000FFFFFFFFFFFFFFFFFFFFFFFFFFFFFFFF09
:10080000FFFFFFFF09490A4A0A4B9B1A03DD043B1D
:10081000C858D050FBDC0849084A0020521A02DDB3
:10082000043A8850FCDC03F061F80000105700081F
:100830000000002030040020300400203807002091
:1008400070B50E4B1A68537A55685C18E4B2A3422F
:100850000ED1537A0A48CB1853720378591AC9B289
:1008600001700020814202D198230130D37070BD05
:1008700006780130EE540133DBB2E8E7940400203F
:1008800098040020FF23F0B5C04C85B02380837905
:100890000700009340780138102801D901F0FEFDCF
:1008A000FFF76AFE1100D405B108F8099F0CFC0D92
:1008B000E80D390BDC0B260C800C4F0A9D0AD90A77
:1008C000080BFC0D830CB878BA888C231D2826D819
:1008D000FFF752FE1E0028001E011802E4028303E7
:1008E0000E04CA04E604F204FA0402050B0514051A
:1008F00022052A0532053A05AA05AA05AA054A05D0
:100900005F057605CC02D8023F058D059605A10549
:10091000B0239F4A5B0351690B435361002323704B
:1009200000F0D8FE152A01D900F081FD1000FFF774
:1009300023FE160023002E007E05390044004F00E0
:100940007E055C006900730080007E057E058D00D9
:100950009A00A700B400C100CE00D800E2009023A6
:10096000DB051A688B490A401A608022D968520355
:100970000A43DA600023D2E790230122DB051968DD
:1009800091431960D9680A43DA600023C7E79023CE
:100990000422DB05196891431960D9680A43DA60BB
:1009A0000023BCE790231022DB05196891431960EE
:1009B000D9680A43DA600023B1E790234022DB05BF
:1009C000196891431960D9680A43DA600023A6E7E1
:1009D0009023DB051A6870490A401A608022D968A2
:1009E000D2040A43DA60002399E79023DB051A68F2
:1009F0006A490A401A608022D96852010A43DA60C3
:100A000000238CE70422664B196891431960D9686A
:100A10000A43DA60002382E79023DB051A68614904
:100A20000A401A608022D968D2050A43DA6000239E
:100A300075E79023DB051A685B490A401A6080223B
:100A4000D968D2020A43DA60002368E79023DB0505
:100A50001A6856490A401A608022D96852000A432F
:100A6000DA6000235BE79023DB051A6850490A40EF
:100A70001A608022D968D2000A43DA6000234EE768
:100A80009023DB051A684B490A401A608022D96816
:100A9000D2010A43DA60002341E79023DB051A689C
:100AA0003D490A401A608022D968D2040A43DA60BC
:100AB000002334E79023DB051A683F490A401A6097
:100AC0008022D96852050A43DA60002327E7012211
:100AD000334B196891431960D9680A43DA600023DF
:100AE0001DE71022354B196891431960D9680A43F4
:100AF000DA60002313E79023DB051A682C490A40CB
:100B00001A608022D968D2000A43DA60002306E71F
:100B1000152A01D900F08EFC1000FFF72DFD1600FC
:100B200021002C008B0451005C0067008B047200D4
:100B30007D00870092008B048B049D00A800B30009
:100B4000BE00C900D400DE00E8009023DB05196870
:100B5000104801401960DA680240DA600023DEE6DE
:100B600090230121DB051A688A431A60DA688A43F8
:100B7000DA600023D3E690230421DB051A688A4358
:100B80001A60DA688A43DA600023C8E600070020AA
:100B900000100240FFFFEFFFFFFFFFFBFFEFFFFF33
:100BA00000040048FFFFFFBFFFFFFBFFFFFEFFFF4A
:100BB000FFFBFFFFFFBFFFFFFFFFFFEF000C004841
:100BC00090231021DB051A688A431A60DA688A4389
:100BD000DA600023A3E690234021DB051A688A43EC
:100BE0001A60DA688A43DA60002398E69023DB050E
:100BF0001968CE4801401960DA680240DA600023C3
:100C00008DE69023DB051968C94801401960DA6850
:100C10000240DA60002382E60421C64B1A688A4348
:100C20001A60DA688A43DA60002378E69023DB05ED
:100C30001968C14801401960DA680240DA6000238F
:100C40006DE69023DB051968BC4801401960DA683D
:100C50000240DA60002362E69023DB051968B84899
:100C600001401960DA680240DA60002357E69023F9
:100C7000DB051968B34801401960DA680240DA60A0
:100C800000234CE69023DB051968AF48014019604A
:100C9000DA680240DA60002341E69023DB05196838
:100CA000A24801401960DA680240DA60002336E6A3
:100CB0009023DB051968A54801401960DA680240F5
:100CC000DA6000232BE601219A4B1A688A431A60E6
:100CD000DA688A43DA60002321E610219C4B1A6807
:100CE0008A431A60DA688A43DA60002317E69023A1
:100CF000DB051968934801401960DA680240DA6040
:100D000000230CE6152A00D997E31000FFF734FC06
:100D100016001F00270095032F0037003F009503A2
:100D20004800510058006100950395036A00730064
:100D30007C0085008E0097009E00A50090228023F5
:100D4000D20511685B030B4313600023E7E5902293
:100D50000123D20511680B4313600023DFE59022C5
:100D60000423D20511680B4313600023D7E59022BA
:100D70001023D20511680B4313600023CFE59022A6
:100D80004023D20511680B4313600023C7E590226E
:100D90008023D2051168DB040B4313600023BEE5FA
:100DA00090228023D20511685B010B43136000235E
:100DB000B5E504235F4A11680B4313600023AEE5D9
:100DC00090228023D2051168DB050B4313600023BA
:100DD000A5E590228023D2051168DB020B43136046
:100DE00000239CE590228023D20511685B000B4311
:100DF0001360002393E590228023D2051168DB0065
:100E00000B43136000238AE590228023D2051168EA
:100E1000DB010B431360002381E590228023D20580
:100E20001168DB040B431360002378E590228023D4
:100E3000D20511685B050B43136000236FE50123A6
:100E40003C4A11680B431360002368E51023404AB5
:100E500011680B431360002361E590228023D205C3
:100E60001168DB000B431360002358E58D23082A2B
:100E700000D054E590224023D20551680B435360C3
:100E800000234CE58D23082A00D048E5902240211C
:100E9000D20553688B435360002340E5152A00D9DF
:100EA000CEE21000FFF768FB16001D002300CC0205
:100EB00029002F003500CC023C0056005B00620088
:100EC000CC02CC0269006F0075007B0082008900B3
:100ED0008E00930090238022DB05D2009A620023CB
:100EE0001DE590230122DB059A62002317E590237C
:100EF0000222DB059A62002311E590230422DB0520
:100F00009A6200230BE590230822DB059A620023F6
:100F100005E590238022DB0592019A620023FEE41E
:100F200090234022DB059A620023F8E4FFFFFFFBD9
:100F3000FFEFFFFF00040048FFFFFFBFFFFFFBFFC5
:100F4000FFFEFFFFFFFBFFFFFFBFFFFFFFFFFFEF06
:100F5000000C00480222CD4B9A620023DFE490236C
:100F60008022DB0512029A620023D8E490238022BB
:100F7000DB0592009A620023D1E490231022DB0566
:100F80009A620023CBE490232022DB059A6200239F
:100F9000C5E490238022DB059A620023BFE49023FE
:100FA0008022DB0592019A620023B8E4902380221C
:100FB000DB05D2019A620023B1E40122B34B9A62AD
:100FC0000023ACE40422B24B9A620023A7E49023EE
:100FD0002022DB059A620023A1E4152A00D932E21F
:100FE0001000FFF7C9FA16001D0023003002290087
:100FF0002F00350030023C00420047004E00300216
:10100000300255005B00610067006E0075007A00D9
:101010007F0090238022DB05D2009A6100237EE4CA
:1010200090230122DB059A61002378E490230222B9
:10103000DB059A61002372E490230422DB059A61A8
:1010400000236CE490230822DB059A61002366E408
:1010500090238022DB0592019A6100235FE49023B4
:101060004022DB059A61002359E40222874B9A61F2
:10107000002354E490238022DB0512029A610023AE
:101080004DE490238022DB0592009A61002346E420
:1010900090231022DB059A61002340E49023202254
:1010A000DB059A6100233AE490238022DB059A61F4
:1010B000002334E490238022DB0592019A6100230F
:1010C0002DE490238022DB05D2019A61002326E4DF
:1010D00001226E4B9A61002321E404226C4B9A6139
:1010E00000231CE490232022DB059A61002316E4F0
:1010F00002236370152A00D9B1E01000FFF722FA2D
:101100000B151EAF273039AF434C545DAFAF67703E
:1011100079828C969EA690238022DB051B69D200E3
:10112000134063800023FFF7FAFB90230122DB05C5
:101130001B69134063800023FFF7F1FB9023022219
:10114000DB051B69134063800023FFF7E8FB902356
:101150000422DB051B69134063800023FFF7DFFBDC
:1011600090230822DB051B69134063800023FFF7EF
:10117000D6FB90238022DB051B699201134063801C
:101180000023FFF7CCFB90234022DB051B691340B3
:1011900063800023FFF7C3FB02223C4B1B69134013
:1011A00063800023FFF7BBFB9023DB051B69DB0B90
:1011B000DB0363800023FFF7B2FB90238022DB0573
:1011C0001B699200134063800023FFF7A8FB902364
:1011D0001022DB051B69134063800023FFF79FFB90
:1011E00090232022DB051B69134063800023FFF757
:1011F00096FB90238022DB051B691340638000234C
:10120000FFF78DFB90238022DB051B6992011340C1
:1012100063800023FFF783FB90238022DB051B699B
:10122000D201134063800023FFF779FB0122174BA3
:101230001B69134063800023FFF771FB0422144BEA
:101240001B69134063800023FFF769FB9023202272
:10125000DB051B69134063800023FFF760FB00235D
:1012600063708D33FFF75BFB80230A4ADB02516911
:101270000B435361054B08491A680A401A60D96844
:10128000064A0A43DA600023FFF749FB00040048DE
:10129000000C004800100240FFFFAAAA00005555AC
:1012A000C84BC9491A680A401A60D968C74A0A4334
:1012B000DA600023FFF733FBC24AC34913680B40CF
:1012C00013600023FFF72BFBBE4AC04B11680B4392
:1012D00013600023FFF723FBBA4912024B69DBB20C
:1012E0001A434A610023FFF71AFBB64B1B691B0A1E
:1012F000A370012363700023FFF711FB8023B44A1E
:101300001B0351690B435361B24AB34B11680B4342
:1013100013600023FFF703FBAE4AAF4BD1680B43CA
:10132000D3600023FFF7FBFAAA4AAC4913680B40CD
:1013300013600023FFF7F3FAA64AA74B11680B438B
:1013400013600023FFF7EBFAA24B5A610023FFF76B
:10135000E6FA012363709F4B1A69A2701B691B0A8E
:10136000E3700023FFF7DBFAC023994ADB025169DF
:101370000B435361934A9A4B11680B4313609022BD
:10138000A023D20511685B030B4313600023FFF712
:10139000C6FA8C4A924BD1680B43D3609023A021AC
:1013A000DB05D86849030143D96011688D480140C5
:1013B00011601A688C490A401A600023FFF7AFFADF
:1013C000FF258048930041692B40884DD200294079
:1013D0000B4343619021C020C905C0004B69024006
:1013E000834803401A434A610023FFF798FA01211A
:1013F000744B1A680A431A6099620023FFF78FFA48
:101400000122704B196891431960D9680A43DA6068
:101410000023FFF784FA6F4B5A610122694B9A61EE
:101420009A620023FFF77BFA0023FFF778FA8D23F7
:10143000FFF775FA8D23FFF772FA8D23FFF76FFA26
:101440008D23FFF76CFA8D23FFF769FABD78BB880F
:10145000052D00D1F1E135D8022D00D185E107D865
:10146000002D00D130E1012D00D13BE196252FE187
:10147000032D00D162E2042DF8D1DBB29825012BB7
:1014800000D025E190225B4BD2051A6006220A218A
:10149000594B1A704B4B594A1360594A1170594AAB
:1014A00001311360584A1170584A13600C22584B8E
:1014B0001A70B023464A5B0351690B43536101F034
:1014C000DDFEAEE1082D00D111E200D9A2E0062D2B
:1014D00000D1CEE1072DC9D101F09CFF902301245A
:1014E000DB051A68384F22431A6010229C61196884
:1014F0000A4304211A60802299611868D2010243CC
:101500001A6080229A6180221868520102431A6090
:1015100040229A6118680143196002219961196893
:101520002B480A431A6008229A61802241691203FB
:101530000A43284942610D68274A2A430A60214A22
:10154000156825431560842594624D6100259461DA
:1015500094624D6180211C68C90521431960802176
:101560000902996280214469C902214341611168DD
:1015700039401160D66815490E43D6601468194E7B
:101580003C401460D4682143D160C0214469C90241
:10159000214341611068124908431060A0201C6873
:1015A000400304431C601468344014601C680E4EF1
:1015B00034401C60D4682143D160DA680243DA60A9
:1015C00086E0C04600040048FFFFAAAA0000555567
:1015D000001002400008004855555555AAAAAAAA6D
:1015E00050550000AFAAFFFFFFFFEBFF03FF000015
:1015F000FFF9000024070020280700201C07002016
:10160000200700202C0700203007002014070020AE
:10161000180700200A2D00D1FAE000D203E1802D46
:1016200000D023E79023012540208026DB0565704C
:1016300098621A68760132431A60C046D2491C6922
:101640001A6804400A401A60DA680A40DA60F02238
:10165000002C36D11A680A401A60DA683243DA6020
:101660001A6994461A690192C0461A690292C046E4
:10167000C0461A690392C046C046C0461F69C046AC
:10168000C046C046C0461E691A680A401A60DA6839
:101690001140D96063462200034212D1019B2A0007
:1016A00003420ED10299023201420AD10399033258
:1016B000014206D10432074203D1D632064200D09D
:1016C000D13AB24B9A70ACE0B14A137001F0A2FE6D
:1016D000AE4C2570AF4B0098A2B2240C5A819C816D
:1016E00005B0F0BD01F096FE9023DB051A682A4391
:1016F0001A6080229D61196852030A431A60802291
:101700000421D2009A621A680A431A6002229A617E
:1017100018680E3202431A604022996119680A4320
:101720001A6008229A6180239B49DB024A699B4D1B
:1017300013439B4A4B6113682B401360D468994B49
:101740001C43D460106828401060D0680343D36005
:1017500080234A691B0313434B61934B934A1968D7
:101760000A431A6000255D61B2E701F053FE902341
:101770000121DB051A6888480A431A601022996122
:101780001968864E0A431A60042240219A611A6839
:101790000A431A6008229A618022996119685201ED
:1017A0000A431A6080224169D2020A437C4942619D
:1017B0000A6832400A60CD687A4A1543CD600C68E9
:1017C00034400C60CC682243CA6080224469120312
:1017D00022434261744A754C15682C4300251460FD
:1017E0005561C0224469D202224342610868704AAE
:1017F00002430A60A0221868520302431A606D482F
:101800004A6902404A615A696B490A405A615FE776
:1018100090238022DB051968D2010A431A608022D6
:101820009A61002554E790238022DB051968D201D4
:101830000A431A6080229A62F3E701F0EBFD9023DD
:101840000121DB051A680A431A60102299611968A0
:101850000A431A60042240219A611A680A431A60F6
:1018600008229A6180221868520102431A60996125
:1018700059E701F0CFFD90230121DB051A68474DA0
:101880000A431A601022996119680A431A600422F7
:101890009A6119683C3211431960082199619A6272
:1018A0009A6180233C49DB024A6913433C4A4B61FD
:1018B00013682B401360D4683A4B1C43D460106803
:1018C00028401060D0680343D36080234A691B031B
:1018D00013434B61344B354A19683848114319603A
:1018E000196801401960D9680A43DA603AE701F0E3
:1018F00091FD90230121DB051A680A431A60042236
:101900009961196811431960196811431960102110
:1019100018680143196040219A611A680A431A60E5
:1019200080229D611868520102431A6099618023E8
:10193000194A1B0351690B435361CBE7DBB2022BFE
:1019400042D00025032B00D1C2E69735012B00D0F1
:10195000BEE68022002510491203486902434A610D
:10196000114A116899431160D1681943D1605168D7
:1019700019435160936111680B431360104B1D7044
:10198000104B1A60A4E6C046FFEFFFFF00070020DF
:10199000080700200060004000100240FFFFAAAAD4
:1019A000000400480000555500080048555555559D
:1019B0005055000003FF0000FFF90000AAAAAAAAE0
:1019C000100700200C070020B023B94A5B035169BF
:1019D00040200B4353619022D2051368B5490B4058
:1019E00013608023D1685B011943D16051680143C2
:1019F0005160906111680B4308211360AE4B197060
:101A0000AE4B1A600DE7BE78F978BD88102E00D174
:101A100010E131D8082E00D108E117D8042E00D1EA
:101A2000E8E00AD8012E00D1B8E0002E00D1ABE0EA
:101A3000022E00D1B6E0A026A9E0062E00D1A8E033
:101A400000D8D3E0280001F05BFAA5E00C2E00D10D
:101A5000F8E008D80A2E00D1DCE000D8D6E0280053
:101A600001F06AF998E00E2E00D1D7E000D8D9E055
:101A7000280001F033FE8FE0242E00D1C4E03FD8CF
:101A8000202E00D1BAE00AD8122E00D1DEE000D21A
:101A9000D4E0132ECFD1280001F0ACF97CE0222E47
:101AA00000D183E000D8ACE0854B9D4202D8802372
:101AB0001B021D43902700F0E5FD6B1CFF339BB21A
:101AC0000193FF057F4B804E5D6132687F4B0002C2
:101AD0001343FF2233607369134018437061C0469B
:101AE0000823BB6200F0CEFD08230135BB61019BDA
:101AF000ADB29D42E6D13368754A134033604BE086
:101B0000842E00D1B3E033D8812E00D1A2E0822E02
:101B100000D1A6E0802E8ED1012190236170DB05DB
:101B20001868644E30401860DA6802203240DA608B
:101B30008022D2009A629961986162484561C046EC
:101B4000C0462DB29A61002D00DA9962C046C046A7
:101B5000C046C046C046C046902280215A4BD2059E
:101B6000C9001B69916201211B0A9161A37013E0F6
:101B7000862E00D186E000D27FE0872E00D05AE783
:101B800001236370534B7BE0280001F005FA2670B7
:101B9000A0E5280001F0DCF90026F8E7280000F0B5
:101BA0008DFFF9E7280001F011F8F5E7454B022217
:101BB0005D6190234448DB059A620668434A090246
:101BC0003243026042692DB2D2B211434161002D0D
:101BD00001DA01229A62C046C04601229A61921837
:101BE0009A6103683A4A13400360D5E7280000F081
:101BF00021FFD1E7280001F05FFDCDE7364B1D70D6
:101C0000CAE7364B1D80C7E7324BF8E7280001F0E2
:101C100021FAC1E7280000F0B7FFBDE7280001F076
:101C20008DFDB9E7280001F0E3F9B5E7280000F0E1
:101C300089FFB1E7280001F039F9ADE7280001F08C
:101C400041F8A9E7280000F0F7FFA5E7280001F018
:101C5000F3F8A1E701232800637001F0ABF8A0704E
:101C60009AE701232800637000F050FFF7E7012393
:101C70002800637000F006FFF1E701236370164B44
:101C80001B7873E702236370144B1B88A3701B0A35
:101C9000E37081E7B878F978BD88AA23062801D9CE
:101CA000FEF73DFEFEF74EFC1C42333A3E4A38003A
:101CB00000100240FFEFFFFF100700200C0700207C
:101CC000FF1F0000000800480004004800005555B0
:101CD000FFFFAAAAA30400208C04002036040020E1
:101CE000FF20CF49AB004A690340CE48ED000240D7
:101CF00013434B619022C021D205C90053690D40A6
:101D0000C9490B401D4355610023FEF708FE002220
:101D1000280000F0CFFCF7E70122F9E7280000F0E7
:101D20000FFEF1E7280000F0E3FDEDE701230021BD
:101D30006370280000F0EEFCA070E5E701216170FF
:101D4000F7E7BA78BB88002A29D0012A44D1B748DE
:101D5000F9784361C020C0011B18B5489BB283428B
:101D600002D89023DB059A62AD4BB24A186809028B
:101D700002431A605A69D2B20A435A61902208217A
:101D8000D2059162C046C046C04691610739916153
:101D90001A68A9490A401A600023FEF7C0FD012114
:101DA000A24A6170536190220420D2059062C02043
:101DB000C0011B189E489BB2834200D89162C04666
:101DC000C046C046C0460121954B1B6991611B0A64
:101DD00003319161A370DFE7AF23FEF7A0FDBD786B
:101DE000022D0BD0032D29D0002D31D10223637099
:101DF00001F0CAFBA070000AE0706AE4BD888F4B56
:101E0000F8781D808E4B8F4A1870884B0002196835
:101E10000A4383491A600E68864A32430A605D614C
:101E20004A69D2B202434A6190220121D2059162ED
:101E30001A6885490A401A6000254AE49023012265
:101E4000DB059A61764A7C4913680B401360F3E71F
:101E5000B025FFF73EFCBA780023012A01D1FEF736
:101E60005EFD9A421FD0B133022A01D0FEF757FD22
:101E700084210125BB886D48194342694161684945
:101E800092B28D618D6242610422802113409022C2
:101E90000902D205002B03D091610023FEF73FFD1C
:101EA0009162FEF73CFD01236370A933A370130018
:101EB000FEF735FDB878BB88042829D8FEF742FB29
:101EC000182803080C00614A13800023FEF727FD41
:101ED000180001F0E1F8F8E790230222DB059A618F
:101EE000C046C046C046C046C046013A9A61ECE7CB
:101EF000902202230421D20563709162C046C0463D
:101F00004A4B1B699161A3709BB21B0AE370DCE72B
:101F1000B223FEF704FDBD78FA78B988112D78D088
:101F200007D8012D4DD0002D0DD0022D5AD082267C
:101F30002DE6212D63D0222D67D0122DF7D102235B
:101F40001020637068E00127414B04261B781020A5
:101F50009F40FA433F4B01921D68AF626B6813408C
:101F60006B6000F084FBAF616B683B436B60FA20F1
:101F7000400000F07CFBFA20AF626B68019A4000E1
:101F800013406B6000F073FBAF616B68013E3B4335
:101F9000B6B26B60002EEAD10436FA2000F067FB7F
:101FA000AF626B68019AFA2013406B6000F05FFB30
:101FB000AF616B68013E3B43B6B26B60002EECD163
:101FC000E5E5234A234B12781E689540B562736895
:101FD0001020AB43736000F04AFBB56173682B437C
:101FE0007360D9E501231A4A637012781A49934045
:101FF000184A9BB21268002002F03AFA2FE6012339
:102000000020637001F0C2FB29E6012310206370F9
:10201000F8E702230020637001F012FC6080BBE54A
:102020000004004803FF0000FFF90000000800481A
:10203000FF1F000000005555FFFFAAAA8A040020D8
:102040008804002055555555AAAAAAAAA004002024
:10205000100700200C07002004000200BB78BA889B
:10206000042B1DD007D8022B1FD024D8012B12D04F
:102070008723FEF754FC072B26D003D8052BF7D176
:10208000BD4B16E0082B24D0802BF1D101F0F6F8DF
:102090000023FEF744FCB94A1278A2706370F7E798
:1020A000B74B1B78A3700123F8E7B44B1A70832257
:1020B000B34B1A70ECE7B14BB14D1A7083232B7000
:1020C00001F04CF92B78EDE7AE4B1A70120A5A70FA
:1020D000DEE7AC4B1A78A2705A78E2709A782271D7
:1020E000DA7862711A79A2715B79E3710623D5E718
:1020F000B878F9780238BA888A23092801D9FEF716
:102100000EFCFEF71FFA050A10151C232F3B404852
:102110009D4B1A800023FEF702FC9B4B1B881B047F
:1021200013439847F6E7FEF723FB0300FEF7F7FBA0
:102130009648036899B213040B430360EAE7934996
:102140000B681B0C1B0413430B60E3E70423637051
:102150008E4B1B681A0AA370E2701A0C1B0E2271B8
:102160006371D7E7022363705300884A1168CB1864
:102170001A88A2701B881B0AE370CBE7834B4900C7
:102180001B68CA52C6E7814953000A68D318022265
:102190000B606270ECE77D4B4900186841181960CC
:1021A0000A80B7E78823FEF7BAFBBB78BA88022B10
:1021B00009D0032B0ED0012B10D11304744A1360E5
:1021C0000023FEF7ACFB72490B681B0C1B04134386
:1021D0000B60F5E701226E4B1A60F1E78323FEF7EF
:1021E0009EFBBA781300303B2F2B1AD8F8780328BF
:1021F00014D8FEF7A7F916180211664B512A00D120
:102200007DE028D8312A57D00FD8002A37D0302A7D
:102210004BD0B423FEF783FB5F4BEFE7B523FEF70C
:102220007EFB5E4BEAE75E4BE8E7332A52D04AD3A7
:10223000502AEED1C022D20022801A7AA270DA7817
:10224000E2705A7A22719A7A62719A78A2715B7CF2
:10225000E371FFF73FFA7F2A00D984E0702A5DD24C
:10226000602A3CD0612A43D0522AD2D180221B88D6
:102270009200A3701B0A2280E370FFF72BFAFF2164
:10228000484BD1540132102AFBD10123434A5B420F
:102290005380434A53803F4A53803F4A5380012230
:1022A000414B1A700023FEF73AFBBA88110AD97223
:1022B0001A730023FEF733FBBA88110A59739A7315
:1022C0000023FEF72CFBBA88110AD9731A74002375
:1022D000FEF725FBBA885A740023FEF720FB802303
:1022E0005B002380BB882F4AD35CA370FFF7F2F911
:1022F00080235B0023802D4B1B68DB78F5E7C02231
:10230000D2002280DA7AA2701A7BE2705A7B2271A4
:102310009A7B6271DA7BA2711B7C99E71F4B38783C
:102320005C68224B1968CB787F2800D9B9E0204837
:10233000009D0570002B0FD000200090982B00D13D
:10234000B5E004E000200090D02B00D1AFE0164BA8
:1023500010301870FF2304E0164B19609023CB70E7
:102360006F330093A3E00720104003283BD8FEF70B
:10237000E9F83D3F2338C046E5040020C4040020AE
:10238000E6040020C50400203404002030040020AE
:102390009C04002060040020740400203804002005
:1023A0004C040020E7040020A40400209004002036
:1023B0009804002094040020494B802A01D2FFF7A2
:1023C00089F9872A16D97032D2B2072A01D9FFF7C4
:1023D00081F900222270FA789A72BA881A80FFF77F
:1023E00079F9404BE9E7B523FEF799FA3E4BE4E76C
:1023F0003E4BE2E7B888F978C6B28D19BE22102D9F
:102400002CDC0432002929D0DD78033AFF2D25D1B8
:102410009D780132FF2D21D10022D7B2B94220D8B8
:10242000334D0022AC464F01013F1F727701000A75
:1024300067449870DA705A729A721A80DA721A7354
:102440005A739A73DA731A745A745F60294B9D1920
:10245000A8540132D3B28B42FAD300222270FFF784
:1024600039F90132B718234D013FEF5DFF2FD4D06A
:10247000C122F3E7BB78002B04D0402B08D0D22335
:10248000FEF74DFA2370BA881B4B1A70FFF722F93A
:1024900080235B002380184B1B7826E78023FEF700
:1024A0003EFAD82B00D04DE780234C68CB70002338
:1024B0004B72CB78902B01D0FFF70CF9712A01D029
:1024C000FFF708F90D4BBA881B6859680A70BA887B
:1024D0005968120A4A705A7A02325A72FFF7FAF8A9
:1024E0006004002074040020380400204C04002004
:1024F000F8040020E7040020A40400209404002035
:10250000F0B51C4D040005A8067868690902C0B240
:102510000843686190200421C00581622900002AD7
:1025200001D101328262FF2500204A692D022A4032
:102530001A43114F4A61C046C046C046C046C04615
:10254000C046C046C046C046C0463A690133120A7A
:1025500022544A69DBB22A4001301A43C0B24A61B0
:10256000B042E8D990230422DB059A61033A9A61CC
:10257000F0BDC0460008004800040048F0B5184C03
:10258000050060690E02C0B2304360618026902071
:10259000F600C00549B28661002901DA0121816295
:1025A000FF2661693602314011436161C046002057
:1025B0000C4FC04639690132090A29546169D2B207
:1025C000314001301143C0B261619842F1D990238A
:1025D0008022DB05D2009A6201229A61F0BDC046DA
:1025E0000008004800040048F0B5174C05000E0034
:1025F00060691F2925D8802131430902C0B20143F7
:10260000616190210420FF26C90588626169360254
:10261000314011436161C04600200C4FC04639690A
:102620000132090A29546169D2B2314001301143A3
:10263000C0B261619842F1D990230422DB059A610E
:10264000F0BDC0B20902DAE7000800480004004803
:10265000002302000002002A04D1002B01D08023B5
:1026600018437047DB43511EDBB20A40F3E70023F7
:10267000800080B2C046C04601339BB29842F9D177
:102680007047FFFF30B50722012409490868450D4E
:1026900043086B404340C50FDBB26B40013A234017
:1026A0004000D2B21843002AF1D10860C0B230BD58
:1026B0009C040020134B10B55861134B13481C6841
:1026C0000902204318605869C0B201435961902142
:1026D0000820C9058862002A01D101328A62C046F9
:1026E000C046C046C046C046C046C046C04690220E
:1026F0000821D2059161073991611A6804490A409D
:102700001A6010BD0008004800040048000055553C
:10271000FFFFAAAA0F4B58619023DB05002901D1C6
:1027200001229A6204229A62C046C046C046C04650
:10273000C046C046C046C046C046C046C046C04669
:10274000C046054908699A61000A033AC0B29A6115
:102750007047C0460008004800040048F7B5040070
:102760000E004D7AC046C046C046C046C046C04670
:10277000C046C046C0460022AA215848FFF79AFF2B
:10278000002255215648FFF795FF24020022202100
:102790005248FFF78FFF23B20193EBB20093337AD5
:1027A000AB4216D28020009B00227372902100025F
:1027B000FFF780FF0022802011000002FFF77AFF60
:1027C00080200022F0210002FFF774FFC0460020A5
:1027D000FEBD444B444A196808200A43FF211A6091
:1027E0005A690A40A02109020A435A619022012134
:1027F000D20590629162C046C046C046C046FF24E2
:10280000906191611A6839492C400A401A60019B15
:10281000009A1C437368A4B2995C20000022FFF761
:1028200049FFC046C046C046C046C046C046C04636
:10283000C046C046C04600212000FFF76BFF0700DE
:10284000C046C046C046C046C046C046C046C04658
:10285000C0467368009A9B5C834217D0C046C0464E
:10286000C046C046C046C046C046C046C04600211D
:102870002000FFF74FFFB8420BD1C046C046C0460C
:10288000C046C046C046C046C046C0460135ADB28F
:1028900083E7C046C046C046C046C046C046C046A4
:1028A000C046C046C046C046C046C046C046C046F8
:1028B000C046C046C046C046C046C046C046C046E8
:1028C000C046C046C046C046C046C046C0460021BD
:1028D0002000FFF71FFF0700C9E7C046AA8A0000D3
:1028E000558500000004004800005555FFFFAAAAC6
:1028F00070B504000D000022AA210F48FFF7DAFE90
:10290000002255210D48FFF7D5FE0022A0210A48DC
:10291000FFF7D0FE002229002000FFF7CBFE0021A8
:102920002000FFF7F7FE0500C04600212000FFF75A
:10293000F1FEA842F3D170BDAA8A000055850000BF
:1029400070B504000D000022AA210F48FFF7B2FE67
:10295000002255210D48FFF7ADFE0022A0210A48B4
:10296000FFF7A8FE002229002000FFF7A3FE0021A8
:102970002000FFF7CFFE0500C04600212000FFF732
:10298000C9FEA842F3D170BD55550000AA2A000027
:10299000C90152080A43FF21F0B585B00293234BC9
:1029A0000500586912B209021140C0B201439024D7
:1029B00059610121E405A1620331A162FF213F2693
:1029C00058690902D2B2084010435861B446002049
:1029D000174F01930391C046C046C046C046C0464B
:1029E000C046C046C0466346396926698908F6086C
:1029F0009E431940314329543E69411C019BC9B291
:102A0000360A6E545969039B01321940D2B2019BB8
:102A1000114359610230029BC0B28342DBD20423CE
:102A2000A361033BA36105B0F0BDC04600080048A8
:102A3000000400480F4B30B59022586180230124D8
:102A4000D205DB0093620C4B94621D680B480902AF
:102A5000284318605869C0B201435961C046082133
:102A60009162C046916119680548014019609461FE
:102A700030BDC0460008004800040048000055551D
:102A8000FFFFAAAA0B4B10B58021586190230122A9
:102A90000424DB05C90099619A629C62C046C04665
:102AA000C046054800699C61000A9962C0B29A61FB
:102AB00010BDC04600080048000400480E4B984274
:102AC00002D880231B0218430C4B0D4A58610D4B52
:102AD0000902186802431A605A69D2B21143596157
:102AE000C04690220821D2059162C04691611A68C1
:102AF00005490A401A607047FF1F0000000800489F
:102B00000000555500040048FFFFAAAA0A4B98424E
:102B100002D880231B021843084B042258619023DB
:102B2000DB059A62C046C046C046C04604490869F3
:102B30009A61000AC0B27047FF1F000000080048F9
:102B40000004004870B504000D000D48AA21FFF7ED
:102B5000B5FF55210B48FFF7B1FFA0210848FFF74B
:102B6000ADFF29002000FFF7A9FF2000FFF7CEFFEF
:102B70000500C0462000FFF7C9FFA842F5D170BD8F
:102B800055150000AA1A000070B504000D000D488C
:102B9000AA21FFF793FF55210B48FFF78FFFA021D4
:102BA0000848FFF78BFF29002000FFF787FF200070
:102BB000FFF7ACFF0500C0462000FFF7A7FFA842C3
:102BC000F5D170BD55150000AA0A00009023DB0561
:102BD00030B51C68134D09022C401C60DA68124C99
:102BE0002A40DA60114A506102229A62104A00B209
:102BF00015682C4314605469E4B22143516180216B
:102C0000C9009961002801DA01209862C046C046D7
:102C100099620121996149189961136805490B402E
:102C2000136030BDFFEFFFFF00005555000800485E
:102C300000040048FFFFAAAAF7B505001C4B01914C
:102C40001E781C4B74001F8820213C19A4B2200060
:102C5000FFF7BCFFAA211848FFF730FFA01B80B286
:102C60001021FFF7B3FF55211448FFF727FF20215C
:102C70002000FFF7ABFFA0210F48FFF71FFF104B0D
:102C8000187846430101BE19C9B2B0B2FFF79EFFE2
:102C900001992800FFF712FF2800FFF737FF040013
:102CA000C0462800FFF732FFA042F5D1F7BDC0466D
:102CB000A30400203604002055150000AA0A0000D5
:102CC0008C04002070B50400B0200E0000020A2120
:102CD000FFF77CFFC0200A210002FFF777FFAA213F
:102CE0001248FFF7EBFE55211148FFF7E7FEA02140
:102CF0000E48FFF7E3FEB0200E4B00021D782900BE
:102D0000FFF764FFC02029000002FFF75FFF3100DA
:102D10002000FFF7D3FE2000FFF7F8FE0500C046B5
:102D20002000FFF7F3FEA842F5D170BD5515000055
:102D3000AA0A00008C040020F8B505000E00194B0B
:102D400002211C88A71CBFB23800FFF73FFFAA2151
:102D50001548FFF7B3FE601C80B20121FFF736FF74
:102D600055211248FFF7AAFE02213800FFF72EFF77
:102D7000A0210D48FFF7A2FE0D4B19786418A0B2F0
:102D8000FFF724FF31002800FFF798FE2800FFF727
:102D9000BDFE0400C0462800FFF7B8FEA042F5D1F2
:102DA000F8BDC0463604002055150000AA0A0000F0
:102DB0008C0400200D4B802258619023D200DB054B
:102DC00000B29A61002801DA01229A62C046C04628
:102DD000C046C046064B802218699023D200DB050E
:102DE0009A620122000AC0B29A6170470008004846
:102DF0000004004870B504000D000D48AA21FFF73B
:102E0000E5FE55210B48FFF7E1FEA0210848FFF73A
:102E1000DDFE29002000FFF7D9FE2000FFF7CAFFE2
:102E20000500C0462000FFF7C5FFA842F5D170BDE0
:102E300055D50000AAAA000070B50400C0200D00FE
:102E400000020121FFF7C2FEAA211548FFF7BEFECE
:102E5000C02000210002FFF7B9FE55211148FFF7FD
:102E6000B5FEC02001210002FFF7B0FEA0210C48F2
:102E7000FFF7ACFEC0200C4B00021978FFF7A6FE4E
:102E800029002000FFF7A2FE2000FFF793FF0500B6
:102E9000C0462000FFF78EFFA842F5D170BDC046A6
:102EA00055950000AAAA00008C04002070B504000B
:102EB0000D001048AA21FFF789FE55210E48FFF7A3
:102EC00085FEA0210B48FFF781FE29002000FFF7B7
:102ED0007DFEA020094B00021978FFF777FE200045
:102EE000FFF768FF0500C0462000FFF763FFA84218
:102EF000F5D170BDAAFA000055F500008C04002041
:102F000070B504000D001048AA21FFF75FFE55219F
:102F10000E48FFF75BFEA0210B48FFF757FE290084
:102F20002000FFF753FE802000210002FFF74EFE35
:102F30002000FFF73FFF0500C0462000FFF73AFFE3
:102F4000A842F5D170BDC04655D50000AAAA000020
:102F50000D4B0E4A58610E4B0902186802431A6065
:102F60005A69D2B21143902259618021D20510686A
:102F70004901014311604021916291611A6805493C
:102F80000A401A607047C0460008004800005555C6
:102F900000040048FFFFAAAA104B114A10B558615F
:102FA0001068104B09020343136053690E4CDBB2E7
:102FB0001943902351618021DB05186849010843BA
:102FC000186040209862186820401860D868014353
:102FD000D960136805490B40136010BD0008004814
:102FE0000004004800005555FFEFFFFFFFFFAAAAAD
:102FF00070B505000E00134B00211C882000FFF760
:10300000E5FDAA211048FFF7C7FF55210F48FFF73C
:10301000C3FFA0210C48FFF7BFFF0D4B19786418C0
:10302000A0B2FFF7D3FD31002800FFF7B5FF28005D
:10303000FFF7C0FE0400C0462800FFF7BBFEA04219
:10304000F5D170BD3604002055550000AA2A0000B5
:103050008C04002070B504000D000D48AA21FFF774
:103060009BFF55210B48FFF797FFA0210848FFF76A
:1030700093FF29002000FFF78FFF2000FFF79AFE43
:103080000500C0462000FFF795FEA842F5D170BDAF
:1030900055550000AA2A0000902270B50225D205DD
:1030A0009561C046C046C046C046C046C0460124E1
:1030B000094B94611E680949314319600849098820
:1030C0005961C04695625861C04694621A680549C4
:1030D0000A401A6070BDC046000800485555555555
:1030E000A0040020AAAAAAAAF0B58BB009920122D6
:1030F00008911100354B02901F78354B1B780493D3
:10310000344B1D68344B1B789940344B019118683F
:10311000334BA9621B789A40029B102B4FD18262DD
:10312000012421002F4B05941B6806932E4B1B781E
:1031300099408BB2210007932C4B1B689C462C4B6B
:103140001B789940002303911900029C202C05D183
:10315000049E059C1E41264236D08261089C202C8C
:103160000FD1002B01D11A4C6354069C2669079C91
:10317000264206D0164C665C059C9C402643144CA7
:103180006654099C013FFFB2002C03D0002F01D1EF
:10319000019CAC616446039E0133DBB2A661A6626A
:1031A000082B05D101310A4BC9B25B5C04930023A3
:1031B000002FCAD1019B8262AB620BB0F0BD029BB3
:1031C000112BADD18261ABE78262C7E7E504002035
:1031D000C50400202C070020300700201C07002019
:1031E00020070020240700202807002014070020C3
:1031F00018070020F7B501221A4B1C781A4B1968E2
:103200001A4B1B789A40102826D18A620126350075
:10321000174B01961B680093164B1B789D400023AB
:10322000AC461D0020280DD1134E019F765D1E4136
:103230003E4215D08A610133DBB2082B02D1002354
:103240000135EDB26646009F013CE4B2BE61BE624C
:10325000002CE7D18A62F7BD1128D7D18A61D5E762
:103260008A62E8E7E50400202C07002030070020F0
:103270001407002018070020C5040020F0B52C4BCF
:1032800085B01B78019301231E00019A1F00964010
:10329000284A1168284A8E62127802921A0002980F
:1032A000824094466046254A126890622448057818
:1032B0002448AF4000689D408762046803941C0066
:1032C000AC402500039C254305604568019CBD4337
:1032D00045609C401D00A54008681C00284308600C
:1032E0004868B04348601068029999408C402100BA
:1032F0000143604611605168814313485160007872
:10330000124A984083401268116899431160D1684D
:103310000B43D36080220E4B1A70002319000D4A14
:1033200013700D4A99540133202BFBD105B0F0BD29
:10333000300700202C070020200700201C07002059
:103340001807002014070020280700202407002069
:10335000E6040020E5040020C504002010B52B4B36
:103360001B78082B4ED013D8294C032B39D006D804
:10337000012B28D0022B2AD0254BEE223AE0062B37
:103380003AD03DD8042BF7D101222021112021E091
:103390000F2B28D008D81E4C0D2B1FD000220E2B2F
:1033A000EAD12021102015E0802B06D0184CFF2BED
:1033B00006D0102BE0D100221FE0FFF75FFF10BD09
:1033C000F0232370FBE72020FFF714FF04E0012225
:1033D00000212020FFF788FE8223F2E7002211005F
:1033E000F7E70122DDE7002220211120FFF77CFE14
:1033F0008222074B1A70E2E7012220210800E9E748
:103400001020E1E71120FFF7F5FEF1E7C4040020EA
:10341000E6040020BC224D4BD203996AF0B50A4362
:103420009A629A6A4A490A409A62B02259695203DA
:103430000A435A6119009023464ADB051278102A84
:1034400003D100221A609A60DA601A6842480124A7
:1034500002401A608022D868D2010243DA601A68FA
:103460003E483F4F02401A608022D8685203024310
:103470000420DA601A68A2431A60DA682243DA602C
:103480001A6882431A60DA680243DA6010221D6803
:1034900095431D60DD682A43DA6040221D6895432C
:1034A0001D60DD682A43DA601A682E4D2A401A60D2
:1034B0008022DD68D2042A43DA601A682A4D2A4045
:1034C0001A608022DD68D2052A43DA601A68274D27
:1034D0002A4080251A60DA68ED022A43DA60244A1D
:1034E0001668A6431660D6683443D4601E683E4012
:1034F0001E60DC683C40DC6080234C691B03234376
:103500004B611C4B1C4C1E681C4F26431E601E68E2
:103510003E401E60DE683443DC604B691D434D61F4
:103520001368174D2B401360D468164B1C43D460AE
:10353000116829401160D1680B43D360136883433D
:103540001360D3681843D060F0BDC046001002403D
:10355000FFFFA1FF08070020FFBFFFFFFFFFEFFFF6
:10356000FFEFFFFFFFFFFFFBFFFFFFBFFFFFFBFFC3
:10357000000400480008004855555555AAAAAAAAB3
:10358000FFFFAAAA000055550D480E4A038810B542
:103590000D49934202D10A7801320A709022042424
:1035A000D205013394620380084B18699461084C7A
:1035B0000B7862691B02D2B2134380B2636110BD03
:1035C0008A040020FFFF0000880400200008004853
:1035D00000040048F7B50D00042701924C7A000260
:1035E00003B2A6B200932B7AB34202D26C720020CF
:1035F000FEBD00986B682043195D80B2019B98471F
:103600006B681A5D094B824205D01A683A431A600A
:1036100002229A61E7E71A680134BA431A60DA684D
:1036200001363A43DA60E4B2B6B2DCE7000400489F
:10363000F7B50D001600FF27000203B24C7A019384
:103640002A7AE3B2A24202D26B720020FEBD2000B1
:103650006A683840D15C019B0134184380B2B0479E
:10366000A4B2EDE7022907D10F4B104A984218D0B7
:10367000904209D1180007E0032906D10A4B0B49F3
:103680000B4A98420BD1080070470429FCD1064B25
:10369000064A984205D006499042F4D0054A88422D
:1036A000E6D11000F0E7C046380400204C040020AA
:1036B000600400207404002070B506000D0005248D
:1036C0003000013CFFF776FBE4B229003000FFF741
:1036D0007DFA6D08002CF3D170BDFFFF70B50400BA
:1036E000A0200D0000020221FFF7E6FFAA211048EA
:1036F000FFF7E4F955210F48FFF7E0F9A0210C4846
:10370000FFF7DCF9A0200C4B00021978FFF7D4FF7B
:1037100029002000FFF7D2F92000FFF7F7F9050094
:10372000C0462000FFF7F2F9A842F5D170BDC046AF
:1037300055150000AA0A00008C04002070B5040092
:10374000C0200D0000020521FFF7B6FFAA210D4899
:10375000FFF73CFA55210C48FFF738FAA021094839
:10376000FFF734FA29002000FFF730FA2000FFF7B6
:1037700021FB0500C0462000FFF71CFBA842F5D145
:1037800070BDC04655550000AAAA0000F7B5012338
:103790000225294F01923A78009105439340042174
:1037A000A020264E2D049BB229433268C00100F0B0
:1037B0005FFE040001283DD13B7809209C40054371
:1037C0007830A3B232682900FF3000F051FE0400C7
:1037D00001282FD13B7832689C402900A3B20020F9
:1037E00000F046FE0400012824D1009B180AFEF7D1
:1037F0002FFF3B7832689C402900A3B200F038FECE
:103800000400012816D16B461878FEF721FF22002C
:103810003B7829009A4093B2326800F029FE019863
:10382000FEF716FF3B7832689C402900A3B200F0F7
:103830001FFE0400E0B2FEBD100700200C070020B0
:10384000F7B501230225274F00903A7801910543EF
:1038500093400421C020244E2D049BB2294332689A
:10386000800100F005FE0400012838D109231D4322
:103870003B78C0209C403268A3B22900400000F091
:10388000F7FD040001282AD13B7832689C402900CA
:10389000A3B2002000F0ECFD040001281FD1019B21
:1038A000180AFEF7D5FE3B7832689C402900A3B287
:1038B00000F0DEFD0400012811D16B461879FEF7F7
:1038C000C7FE22003B789A4093B2009A1443092223
:1038D000E1B209041143326800F0CAFD0400A0B24D
:1038E000FEBDC046100700200C070020C74BC84A89
:1038F000F0B51A60C74A8BB01A6002225A60A02243
:1039000012019A600493049BDB68002BFBD1902288
:10391000049BC14912031960C04B186802431A6026
:1039200080220991920219681142FCD00122596843
:103930000A435A608022596852020A435A60802220
:10394000596852030A435A608022196852040A4394
:103950001A608022920419681142FCD01121B04AE9
:10396000B04C11605A680E398A43110002220A4392
:103970005A608022196B0A431A638022D9691204A3
:103980000A43DA61A84BE381BC231B689847A74B25
:103990006382A74B238262B6FFF73CFDF022A54B62
:1039A0001A70049B099AA44E1A60327820231100E1
:1039B0009943D2291BD1A149A148C978C3780224CF
:1039C000FF2904D1FF3B1C00631E9C41E4B29D4BC8
:1039D000DB78FF2B00D003249B4BDB78FF2B00D040
:1039E00004249A4B9A4F1C703860D22A56D03378F0
:1039F000F22B05D10022023B3370954B1B68DA7025
:103A00003578D02D00D0D6E1914E3068C378802B28
:103A100000D0D0E18D4B1978FFF724FE00233060F1
:103A2000C570068804004372C07AF5B210382028A9
:103A300000D9BEE1FCF7A0FD12014A018D01910100
:103A4000BD01BD01BD01BD01BD01BD01BD01BD0186
:103A5000BD01BD01BD01BD01350042005000550052
:103A6000580062006900A600BC00C400BD01BD0191
:103A7000BD01BD01BD01BD01CB002100FFF7F2FD7D
:103A800001230135EDB2A542F7D3002B00D03860F9
:103A900080223B68DA70D0233370A8E70023012529
:103AA000F1E7E17B0F2900D9A6E109013143237A2F
:103AB000A278C9B26068FEF761FD0BE03C23E17BB0
:103AC0000A009A4300D097E1237AA27829436068DC
:103AD000FEF78AFD607262E0237AA278E17B2943D7
:103AE000E8E7E17B3F23EBE7227AE17BA3780092D2
:103AF000002229436068FEF703FDEBE7E17B227AB1
:103B0000A378294300920122F4E7524BE17B5869E4
:103B100029430E02C0B230436568A278277A586103
:103B2000902004266031C005C9B286621E001F299C
:103B300001D801218162FF2059690002014011432F
:103B40005961C046444900238C46C046C046C04621
:103B5000C046C046C046C046614609690132090AEE
:103B6000E9547169D2B2014001331143DBB2716192
:103B70009F42EAD290220421D205916103399161DA
:103B800063720CE00025267A67687608FFF7FCFC74
:103B90000135EDB238800237AE42F7D265722C4B58
:103BA0001B6819889A7A52181A80D822DA7002E1B2
:103BB000E17B237AA27829436068FEF7E9FE89E772
:103BC000E17B237A29430131A278FF31F4E7A07821
:103BD0002D0228436668277AFFF75EFA1D4A902077
:103BE000002304259446C0058562C046C04662464F
:103BF000116985618AB2120AF2545A1C0233D2B298
:103C0000DBB2B1549F42EFD2BAE7C0460030004069
:103C1000CCCC000055550000AAAA000000100240BC
:103C200000200240006000403CA5FFFF4108000862
:103C300085080008E6040020A40400204C040020AD
:103C4000380400206004002074040020A204002036
:103C5000900400200008004800040048E37B1E2B6D
:103C60000BD1C020B6092233F1B200029D43FEF70A
:103C7000ADFF237AA278802131E71C2B0FD1A02041
:103C80008121C001FEF7A2FF8020F609F1B20002F7
:103C9000FEF79CFFA0200021C001FEF797FF8021C6
:103CA000E27B49421F2A05D00D43EDB2237AA27868
:103CB0002900FFE67022A02095430D432188C00112
:103CC0000909C9B2EDB2FEF781FFEFE7E37BFE2BF6
:103CD00000D064E77609F1B2C348FEF7EFFE1F217A
:103CE000636829409C46C14B09025A69A678D2B242
:103CF0000A43277A80215A619022C900D205916136
:103D00000121FF209162033191625A690002024051
:103D100032435A61C0460022B54D0290C04660460B
:103D200029690136090A815459690298F6B201409D
:103D300001323143D2B259619742EFD2902304212C
:103D4000DB0599618021C900996201219961627244
:103D500025E7237AA2786021C1E6E37B002B20D1FE
:103D60008033F6091D43F3B20393FF20039BA04960
:103D70009B004A6903409F48024013434B61C020A7
:103D80009021039BC905C000DB004A6903409A48A3
:103D9000024013434B61227AA3782900009200224B
:103DA000A8E6012BE1D140217604760E3143039140
:103DB000DBE7C323E370914B1D78F02D00D037E390
:103DC0008F4E3468E378982B00D031E38D4B200080
:103DD0001978FFF747FC00233060C370E07AE57084
:103DE00010382678042800D920E3FCF7C5FB07002B
:103DF00002029002BB02F600C423DBE7E37B002B48
:103E000006D130008038C0B27F4A2100FFF7E2FBC4
:103E1000E37B012B06D130008038C0B27B4A210001
:103E2000FFF706FCE37B032B06D130008038C0B2DD
:103E3000774A2100FFF7FCFBE37B042B06D130001F
:103E40008038C0B2734A2100FFF7C4FBE37B0A2B22
:103E500006D130008038C0B26F4A2100FFF7E8FB7E
:103E6000E37BFD2B15D13F20238830409B09059330
:103E70006B4680261B7D06430793677ABBB202938D
:103E800033021BB20893237A029A934200D3CFE005
:103E90006772E37B1E2B06D130008038C0B25F4AC8
:103EA0002100FFF797FBE37B0C2B17D11F2030403D
:103EB00080260643C0202588A5216D09EDB2C001EA
:103EC000FEF784FE29005648FEF780FE677A350229
:103ED0003D43237ABB4200D3F2E06772E37B1C2BA5
:103EE0003BD1A02023888121DB09DBB2C0010593EF
:103EF000FEF76CFE802005990002FEF767FEA02009
:103F00005421C001FEF762FE677AAA21BBB2454880
:103F10000293FEF75BFE55214348FEF757FE202132
:103F20004048FEF753FE802333431B021BB2079326
:103F3000237A029A934200D3DFE08020902100028E
:103F40006772FEF743FE802000210002FEF73EFE6E
:103F50008020F0210002FEF739FEE37B1F2B32D1D7
:103F6000A020218851330909C9B2C0019E43FEF740
:103F70002DFE677AAA21BBB22A480293FEF726FEDD
:103F800055212948FEF722FE20212648FEF71EFE75
:103F900080235B4233435BB21B020693237A029A6F
:103FA000934200D3F1E08020902100026772FEF777
:103FB0000DFE802000210002FEF708FE8020F02187
:103FC0000002FEF703FEE37B6F2B06D13000803842
:103FD000C0B2164A2100FFF7FDFAF4232288E370ED
:103FE000A37A9B18238023E2FF3F000000080048CB
:103FF0000004004803FF0000FFF90000A4040020B3
:1040000090040020A2040020553000083D3700082D
:10401000F12F0008012F0008AD2E0008392E0008EE
:10402000FFFF0000AA8A000055850000F52D00085A
:104030000021BB48FEF7CAFDAA21BA48FEF788FF57
:104040005521B948FEF784FFA021B648FEF780FF4E
:104050006B46187DB54B0799C01880B2FEF7B6FDC8
:10406000089D63683D43ADB2D95D2800FEF770FF3F
:10407000C0462800FEF79EFE06902800FEF79AFE36
:10408000069B8342F4D163680699DA5DA84B8A42A5
:104090000FD1029A1968013292B20292042291431E
:1040A0001960D96801370A43DA600222FFB29A62C6
:1040B000E9E6042219680A431A6002229A61E2E6DC
:1040C000AA219C48FEF782FD55219B48FEF77EFD04
:1040D000A0219848FEF77AFD63682800D95DFEF7B5
:1040E00075FDC0462800FEF765FE02902800FEF729
:1040F00061FE029B8342F4D1EBE6A0205421C00173
:10410000FEF764FD079DA0213D43ADB22800FEF7F8
:104110005DFD63682800D95DFEF758FDC0462800A4
:10412000FEF748FE06902800FEF744FE069B8342F9
:10413000F4D16368069ADB5D7D4D93420FD1029BFB
:104140002A6801339BB2029304239A432A60EA68E7
:1041500001371343EB600223FFB2AB62E8E6A02015
:104160008121C001FEF732FD802005990002FEF793
:104170002DFDA0205421C001FEF728FD04232A684C
:1041800013432B600223AB61D2E6069DA0213D4381
:10419000ADB22800FEF71AFD63682800D95DFEF76E
:1041A00015FDC0462800FEF705FE05902800FEF725
:1041B00001FE059B8342F4D163680599DA5D5C4B8F
:1041C0008A420FD10421029A0137013292B202923F
:1041D0001A68FFB28A431A60DA680A43DA60022278
:1041E0009A62DBE604211A680A431A6002229A6185
:1041F000D4E6E37B002B04D1504A21003000FFF7C6
:1042000017FAE37B012B04D14D4A21003000FFF760
:104210000FFAE37B022B04D14A4A21003000FFF75A
:1042200007FAE37B042B04D1474A21003000FFF753
:10423000FFF9E37B0A2B04D1444A21003000FFF749
:10424000F7F9E37B0B2B04D1414A21003000FFF743
:10425000EFF9E37BFE2B00D0BFE621883D484909FA
:10426000C9B2FEF72BFCAA213B48657AFEF7E2FBB8
:1042700055213A48FEF7DEFB37482021FEF7DAFBEE
:104280001F2030400302AFB20593237ABB420DD208
:10429000657290210020FEF7CDFB00210800FEF79B
:1042A000C9FBF0210020FEF7C5FB96E6059EA02184
:1042B0002E433000FEF7BEFB63683000595DFEF709
:1042C000B9FBC0463000FEF7DDFB02903000FEF780
:1042D000D9FB029B8342F4D1636802995A5D144B67
:1042E0008A420DD104211A6801358A431A60DA68BE
:1042F00001370A43DA600222EDB2BFB29A62C4E724
:1043000004211A680A431A6002229A61BDE730004C
:104310006030134A2100C0B2FFF78AF95DE6C0465B
:1043200069FD000055550000AA2A000069FDFFFF45
:104330000004004855D50000AAAA0000892B0008F7
:10434000DD360008392D0008452B0008C52C000873
:10435000392C0008FF3F0000AA0A000055050000A4
:10436000CD2B0008E37B042B06D130008038C0B28F
:10437000364A2100FFF75CF9E37B052B04D1334A71
:1043800021003000FFF754F9E37B062B06D1300003
:104390008038C0B22E4A2100FFF74AF9E37B072B91
:1043A00004D12B4A21003000FFF742F9E37B002BB8
:1043B0001CD1FF2280331E4323882648DB09DBB251
:1043C0009D0041692A40244DDB0029400A43426197
:1043D0009022C020D205C000516903401F4801400F
:1043E0000B43536121003000FEF7B8F9E37B012B4A
:1043F00000D0F2E52388174A5B04580E402303439C
:10440000FF209B0051690340134801400B4390215A
:104410005361C9054B69114A30001A4080239B0043
:1044200013434B612100FEF799F9D6E5C323E370EE
:104430000B4B1B78F02B01D1FFF7B3FA832B01D084
:10444000FFF7AFFAFEF78AFFFFF7ABFA4129000842
:10445000F12800080004004803FF0000FFF90000F5
:10446000E6040020FFFFFFFFFFFFFFFFFFFFFFFF4E
:10447000F0B5474680B4061C081C000C102801D576
:10448000162700E004270007000F8046FF200140A8
:104490005468251C1D439C43F60313850AD5C0466A
:1044A000C046C046C046C046C046C046948013833E
:1044B000958002E0012000F081F801390AD4381C0F
:1044C00000F07CF8C046948013839580C046C046B7
:1044D0007600E2E7381C013800F070F8948013830E
:1044E0009580042000F06AF8108A184001D0FF205F
:1044F00061E0C046C046C046C046C046C046948043
:104500009580108A184055D001200226B04552D01F
:104510000921168A1E40FCD1012000F04FF894803A
:10452000C0469580C04603E0C046C046C046C0466F
:10453000948095807600108A1840EFF30080400048
:10454000C00F0643381C023800F038F8948095807C
:10455000022000F033F80139EAD513859480012058
:1045600000F02CF813839580301C802102239940A1
:104570000E401BD1002341085E4149085E414908B5
:104580005E4149085E4149085E4149085E4149086B
:104590005E4149085E4149085E41760808D34008FB
:1045A000FF21084048400002013004E00E2002E0F4
:1045B000092000E0002080BCB846F0BD0138FDD1E4
:1045C0007047C04603685A0003D45B005B08C018FC
:1045D0007047802212061343F9E7C046F0B55746EC
:1045E0004E46DE464546E0B5814683B092460029F8
:1045F00025D04B1E9B46002701935B46FB18DC0F22
:10460000E4184B466410E5005E193000FFF7DAFF4E
:10461000019B8046A3420BD0280008304844FFF796
:10462000D1FFD04506D80138504509D2671CE4E7D0
:10463000504505D9A74202D0631E9B46DDE7002600
:10464000300003B03CBC90469946A246AB46F0BD54
:10465000012809D0022805D0002801D00020704789
:104660000248FCE70248FAE70248F8E7454D00082F
:104670005D4D0008514D000830B5234B83B0050057
:104680008C1E002B26D001A9200000E000BF0028CE
:104690001CD001992200FFF7A1FF041E16D0FFF7DE
:1046A00091FF6368A864012B2AD0201D002B23DB17
:1046B000FFF788FF0023E8642B650368002B0FDBFE
:1046C000FFF780FF2861002003B030BD00230920E0
:1046D0002B61F9E70D480E49091AC9100191D9E774
:1046E0001801000FFFF7B4FF2861431E984108230B
:1046F000404298430930E7E70123E8642B65DCE793
:10470000002305202B61DFE7000000004056000871
:1047100010570008036810B50400DA0705D44830C4
:104720009B070ED500F06CFC23685A070ED51A07BC
:1047300013D5DB0604D42000D130FF3000F06CFC30
:1047400010BD00F059FC23685A07F0D42000D03087
:1047500000F05AFC23681A07EBD420005130FF30D8
:1047600000F056FC2368E4E70368002B00D01B1818
:1047700018007047092070477047C04670B50400A4
:104780000D0008E02B6C2A006361210001202369E1
:104790009847082807D1296C2000FFF76DFF0028F3
:1047A000F0D000F083FE0728FBD10020296CFFF732
:1047B000E3FF281D00F00AFCF0B5CE46474680B561
:1047C000C3682E4C9846A544836906001400043142
:1047D000402205A8994600F071FE002304AD049321
:1047E00023E0F0222B6C5200736129007CA800F0BA
:1047F00065FE7CAA31003369200098478A9B070038
:104800006B6403934B460095019332003300210003
:104810000120C04700281FD1F0227CA952002800A7
:1048200000F04CFE0024082F1FD1296C3000FFF748
:1048300023FF611E8C41070009340028D1D0AB6BE7
:1048400010216B644B4621430193009533003200E5
:104850000120C047002800D009273800F5239B001D
:104860009D440CBC90469946F0BD072FF4D1200022
:10487000296CFFF781FF05A800F0A8FB2CFCFFFFC7
:10488000406C704770B5CB6BFAB00B6404000E003F
:104890004022043103A800F011FE01235B42029381
:1048A00006E002AA210023699847050008280AD1DA
:1048B000129B200019000193FFF7DEFE0028F0D0C4
:1048C00009207AB070BD02A8FFF724FF062DF7D1AA
:1048D00031002000FFF752FF10B58261DA6BC16032
:1048E0001A6419000022FFF767FF10BD436970B515
:1048F0000B64C36804000D00002B15D10A00236966
:10490000010002209847072807D0082803D1290072
:104910002000FFF733FF00F0C9FD0020296CFFF7EE
:104920002BFF281D00F052FB0122FFF745FF00F08E
:10493000BDFDC046C36810B5002B05D0CB6B00226F
:104940000B64FFF739FF10BDFFF79CFFFBE7C04684
:104950007047C046836810B5002B02D001000120CB
:10496000984710BD012906D0002906D0033902203E
:10497000012900D970470120FCE7002B08D10F2A3C
:1049800006D8920082185268009B00201A60F1E756
:104990000220EFE700B585B003AB0A0000930021C9
:1049A0000023FFF7DFFF039805B000BD012906D003
:1049B000002906D003390220012900D970470120BF
:1049C000FCE7002B08D10F2A06D8009B92001B6839
:1049D000821853600020F1E70220EFE700B585B0B0
:1049E00003AB039200930A0000230021FFF7DEFFD0
:1049F00005B000BD70B51A4CD36BA5441364060016
:104A00000D0019A8111D402200F058FD01235B4242
:104A1000189314E00C2118A802AAFFF7DFFF290061
:104A200018A8B047002812D1069B18AA02A908307E
:104A300001939847040005280AD0092807D0289B2D
:104A400002A819000193FFF717FE0028E2D00924FD
:104A500018A8FFF75FFE200090239B009D4470BDC7
:104A6000C0FDFFFFF0B5DE4657464E464546E0B571
:104A7000160003220D0011008BB01F000193EB6C98
:104A800001401C1D009107A91B688B460894002F4C
:104A90006BD01A0C1B045946079302230B72FD338B
:104AA00013409B004A72E418009B022B00D1AC6BB0
:104AB0002B6DDB0747D40023059308330340029393
:104AC0002768002F00D112E1019B022B49D0638897
:104AD000278898460434012340469A469843AB6C95
:104AE0000F21994681443000FFF754FF0021814592
:104AF00006D839005346994349448842894149427E
:104B000043465A0002231340012217403B43012B26
:104B10003AD0002B30D0022B1BD12368009A5F00C3
:104B20007F08002A67D1002906D0029A002A00D106
:104B30007CE0002F00D1A9E0002B00DA043401371B
:104B4000BF00E419BCE75946300000F00BFB002819
:104B500010D009200BB03CBC90469946A246AB460B
:104B6000F0BD636808349846B5E71B0207935B46BF
:104B70001A8199E70820EDE7009B002B02D000295D
:104B800000D08DE004349BE7009B002B1AD1002954
:104B900016D02368DF0F63689A1CDAD02A005832D7
:104BA0000692013300D1BDE0201DFFF7DDFD06AB0D
:104BB00001003A00280000E000BF002800D082E099
:104BC00008347DE70D2130002F6AFFF7E3FE8742AE
:104BD000F6D1AB6A9C42F3D12000FFF7F3FC0F2122
:104BE00002003000FFF7FAFE30002A000021FFF734
:104BF000F5FE0720AEE72B6A0D2130009846FFF73F
:104C0000C9FE804501D0236896E7AB6A9C42FAD181
:104C10000023EB6204332B63231DAF626B632368B5
:104C2000002B00DA86E00123059388E7002F2DD0C2
:104C300058239C46AC4463460393231D99460023A6
:104C4000984606AB220004933B004C464746B246CA
:104C500098462E00914603E004342F00454542D08B
:104C6000039B20000693FFF77FFD049B01000022B9
:104C700030007D1C00E000BF0028EDD04346B84660
:104C800035004C4656461F009845BCD10D213000DA
:104C9000FFF780FE069B28626B62AC62062059E734
:104CA0002000FFF78FFC04340700AC63280000E00D
:104CB00000BF002800D14CE730003A000F21FFF779
:104CC0008DFE072046E707000D213000FFF762FE4A
:104CD0002862022F2BD1069BEB622B002C336B62D8
:104CE000AC62062036E735004C465646CEE75946BC
:104CF000300000F037FA002800D02AE7059B002B8F
:104D000000D137E70F213000FFF744FE0E210200EB
:104D10003000FFF763FE3000094A0F21FFF75EFE07
:104D2000072017E70D213000FFF734FE2862069BAD
:104D30006B62D5E738000130800020184DE7C0468F
:104D40000000000010B50023FFF78CFE10BDC04628
:104D500010B50123FFF786FE10BDC04610B5022333
:104D6000FFF780FE10BDC046F0B5CE46474680B581
:104D70000500C3B014001E00012955D000294BD0F6
:104D8000032922D0042949D1002B47D1102A45D824
:104D9000102203681A4200D0F1E020AF380000F082
:104DA0003DF900230120A96B02009A40144203D070
:104DB0000E689A00BE5004310133042BF4D1380040
:104DC000A96300F029F9002029E0032B26D114045F
:104DD000230C160C9846F318102B1FD808220368D2
:104DE0001A4200D098E020AF380000F013F9424694
:104DF000AB6BF6001C00002A08D0D400F21A1C1974
:104E0000BA181968D15004339C42FAD1AC63380007
:104E100000F0FEF8002002E0002B24D0022043B076
:104E20000CBC90469946F0BD130C14049846240C13
:104E3000012E2ED0052EF1D11B19202BEED8424683
:104E40000F2A70D9A146002C7ED1AA6B4346AA63D3
:104E50000F2B00D89AE04B46002BDBD0684600F0C1
:104E6000D3F80020DBE700231004A96B000C013607
:104E700032009A40104204D00F689A00AA18576076
:104E800004310133102BF3D10020A304C7D4A9634C
:104E9000C5E71B19102BC1D843460F2BBED82B6872
:104EA0001E4206D00322280093432B60483000F0B6
:104EB000A5F820AF380000F0A1F8AA6B002C24D090
:104EC0004346DB00FF180023994664000023A4003A
:104ED000D158F95004339C42FAD14B4612196F460F
:104EE000002B0FD04046102800D210204B46D9008E
:104EF00000231038C0003818D458C45004339942E5
:104F0000FAD15218012EA1D120AF04323800AA6381
:104F100000F072F8002082E7934303605130FF30C5
:104F200000F078F85FE7102B3BD9102252429146EF
:104F300099442B68194208D0022228008B4313435E
:104F40002B60483000F05EF82B6804221A4221D111
:104F500043460F2B03D820AF380000F053F86F46BC
:104F6000380000F053F810244346AA6BE41A002CD2
:104F7000B8DD434620AFDB006400FF18A6E793438B
:104F80000360D130FF3000F049F806E720A800F0B8
:104F900037F860E7280093432B60D03000F036F8F4
:104FA000D6E72B680B4207D0022228008B4313431D
:104FB0002B60483000F026F820AF380000F022F8CF
:104FC000A146AA6B002C00D07AE73FE7011C3431E0
:104FD00038C9043B9C461D60A646011C20313CC9D3
:104FE00090469946A246AB46011C0831FCC941686F
:104FF0000068E54600BDC0467047C0467047C046E1
:105000007047C0467047C0467047C0467047C046AC
:105010007047C0467047C0467047C0467047C0469C
:1050200001B401A801B585B0FFB408A841464A46BD
:1050300053465C4665463EC001A83EC80F980090A6
:1050400000230CB401A9FFF71DFC109B12B01847F8
:1050500001B401A801B585B0FFB408A841464A468D
:1050600053465C4665463EC001A83EC80F98009076
:1050700000230CB401A9FFF739FC109B12B01847AC
:1050800001B401A801B585B0FFB408A841464A465D
:1050900053465C4665463EC001A83EC80F98009046
:1050A00000230CB401A9FFF745FC109B12B0184770
:1050B00001B401A801B585B0FFB408A841464A462D
:1050C00053465C4665463EC001A83EC80F98009016
:1050D00000230CB401ABFFF7FFFB109B12B0184785
:1050E00001B401A801B585B0FFB408A841464A46FD
:1050F00053465C4665463EC001A83EC80F980090E6
:1051000000230CB401AAFFF775FC109B12B01847DE
:10511000027A0300002A0BD1427A002A0FD0013A0A
:1051200042724268111D416003211268017202E05F
:10513000013A02720268100E12021A607047B02023
:10514000FCE7C04600B585B003AB00930C220023FA
:105150000021FFF707FC039805B000BD10B5FFF76D
:10516000F1FF10BDF0B557464E464546DE460023DA
:10517000E0B587B003930F339846083B99468023E8
:105180001B0306000F009A463800FFF7C1FF04001A
:10519000B02800D1C3E003062AD50300424693435A
:1051A000DBB2802B00D171E0902B3DD0A02B00D141
:1051B00085E0B02B50D0C02B00D196E003004A46CA
:1051C0009343DBB2D02B0AD15346024001321A433B
:1051D000052301213000FFF7C7FD0028D4D00924A2
:1051E000200007B03CBC90469946A246AB46F0BDB5
:1051F000FF23820013401D1D05AB9B4600930D222B
:10520000002300213000FFF7ADFB630620D4059B8F
:105210009C46654405955B460D22009300210023C2
:105220003000FFF7C3FBAFE7833B03400D2BD6D025
:1052300005AD02400095002300213000FFF792FBEE
:10524000009500230D2200213000FFF7AFFB9BE704
:10525000059B5D1B0595DEE7B12874D0B22800D10F
:10526000CFE0B32800D184E0FC230340B42BB6D0B8
:105270004A465346024001321A43012101233000BD
:10528000FFF772FD002800D17EE7A8E7040238008E
:10529000FFF73EFF802520432D02A8429FD0040146
:1052A0000005020C002300213000FFF75DFD0028FF
:1052B00095D12C4200D167E70123039364E7FF23D4
:1052C0004A461B011900824311410A001A40030794
:1052D00002D58023DB011A43002300213000FFF7B1
:1052E00043FD002800D14FE779E7C6284CD0C728F6
:1052F0005ED003004A469343DBB2C02B6DD0C82872
:1053000072D0C92800D06AE73800FFF701FFF02308
:1053100002031B03134042460240013257E7039B3E
:105320000024002B00D05BE705AD00950E22002184
:105330003000FFF717FB009500230F2200213000FB
:10534000FFF734FB4CE73800FFF7E2FE002800D1FE
:1053500045E7030042469343DBB2002B00D03EE713
:10536000020000213000FFF7FFFC002800D10BE70E
:1053700035E73800FFF7CCFEF02302031B03134090
:1053800042460240013277E73800FFF7C1FEF023C2
:1053900002031B0313404246024001321A43032317
:1053A00003213000FFF7E0FC002800D1ECE616E70F
:1053B0003800FFF7ADFE021E00D110E703004146A2
:1053C0008B43DBB2002B00D009E704213000FFF74C
:1053D000CBFC002800D1D7E601E74346A0221C40C1
:1053E000013412032243DAE73800FFF791FE434607
:1053F00002009A43D2B21032184012030130024325
:10540000E6E605AB00939B460D2200230021300009
:10541000FFF7A8FA3800FFF77BFE030618D57F25B3
:10542000B03C059B2840A0409C4660440590380055
:105430000734FFF76DFE0306F3D481217F23890033
:1054400003408C46A340059A62449B180593E2E60C
:105450000224F2E7030000B5DB6C85B05A6808004F
:10546000120201921A0001A908324A6003220A724C
:10547000DB794B72FFF776FE05B000BD10B5FFF784
:105480006DFE806C10BDC04610B5FFF767FEC26CA4
:10549000D3799B000833D01810BDC04610B500F07A
:1054A00005F8C04610B5FFF7F9FFC04610B5062055
:1054B00000F076F8012000F0A5F8C046F0B50F2AFC
:1054C00037D90D0005430C000300AD0735D1150099
:1054D000103D2D092E013618103627681F606768A9
:1054E0005F60A7689F60E7681034DF601033B342E5
:1054F000F3D10F2401352D01491914404519032C0E
:105500001DD90023CE58EE500433E61A032EF9D8E5
:105510000323043CA4080134A4001A402D190919DE
:10552000002A05D00023CC5CEC5401339342FAD11D
:10553000F0BD0500002AF5D1FAE70500F2E72200E8
:10554000F8E7C04670B505000C001F2922D8B72324
:105550009B00C358002B0ED08A009B181A68002AA3
:1055600009D0012A10D0511C10D000212000196050
:105570009047002070BD280000F030F822000100A4
:10558000280000F017F8F5E70020F3E71623036082
:105590000120EFE71623036001204042EAE7C046FE
:1055A00010B5034B01001868FFF7CCFF10BDC046D3
:1055B00000000020002370B5074C05000800110012
:1055C000236000F017F8431C00D070BD2368002B47
:1055D000FBD02B60F9E7C0463407002010B500F07F
:1055E00001F810BD58220120014B40421A6070475B
:1055F0003407002058220120014B40421A607047B6
:1056000034070020FEE7C046F8B5C046F8B5C046EE
:1056100074B20181B0AB308000000000800A0181CB
:10562000B0B0ABF0000000003F020181B0AB3080B1
:105630000000000080060181B0B0ABF00000000067
:1056400030EEFF7FB0B0B0807CEFFF7F0100000044
:1056500028F0FF7FB0A90280BCF0FF7FB0B0A88027
:1056600008F1FF7F0100000014F1FF7FB0B0AA80B5
:1056700048F1FF7F9CFFFF7F08F2FF7F01000000E1
:1056800004F2FF7FAA3F398050F2FF7FB0B0A880BC
:105690005CF2FF7FB0B0AA809CF2FF7FB0B0A88020
:1056A000B0F2FF7F01000000ACF2FF7FB0B0A88035
:1056B000B4F2FF7F010000003CF3FF7FAA0FB2802D
:1056C000A4F3FF7F58FFFF7F7CF6FF7FB0B0A88078
:1056D00098F6FF7F54FFFF7FF4F8FF7F0100000082
:1056E00064FAFF7F0084048074FAFF7FB0B0A88062
:1056F00074FAFF7F40FFFF7F5CFDFF7F0084048022
:105700007CFDFF7FB0B0A88094FDFF7F010000000A
:10571000080000200000000000000000F40200204B
:105720005C030020C4030020000000000000000013
:105730000000000000000000000000000000000069
:105740000000000000000000000000000000000059
:105750000000000000000000000000000000000049
:105760000000000000000000000000000000000039
:105770000000000000000000000000000000000029
:105780000000000000000000000000000000000019
:105790000000000000000000000000000000000009
:1057A00000000000000000000000000000000000F9
:1057B00000000000000000000000000000000000E9
:1057C00001000000000000000E33CDAB34126DE686
:1057D000ECDE05000B0000000000000000000000EF
:1057E00000000000000000000000000000000000B9
:1057F00000000000000000000000000000000000A9
:105800000000000000000000000000000000000098
:105810000000000000000000000000000000000088
:0400000508000805E2
:00000001FF
